:020000040000FA
:10000000BC280400000000003C2400003C24000048
:100010003C2400003C2400003C2400003C24000060
:100020003C2400003C2400003C2400003C24000050
:100030003C240000582400003C2400003C24000024
:100040003C2400003C2400003C2400003C24000030
:100050003C2400002E2600003C2400003C2400002C
:100060003C2400003C2400003C2400003C24000010
:100070003C2400003C2400003C2400003C24000000
:100080003C2400003C2400003C2400003C240000F0
:100090003C2400003C2400003C2400003C240000E0
:1000A0003C2400003C2400003C2400003C240000D0
:1000B0003C2400003C2400003C2400003C240000C0
:1000C0003C2400003C2400003C2400003C240000B0
:1000D0003C2400003C2400003C2400003C240000A0
:1000E0003C2400003C2400003C2400003C24000090
:1000F0003C2400003C2400003C2400003C24000080
:100100003C2400003C2400003C2400003C2400006F
:100110003C2400003C2400003C2400003C2400005F
:100120003C2400003C2400003C2400003C2400004F
:100130003C2400003C2400003C2400003C2400003F
:100140003C2400003C2400003C2400003C2400002F
:100150003C2400003C2400003C2400003C2400001F
:100160003C2400003C2400003C2400003C2400000F
:100170003C2400003C2400003C2400003C240000FF
:100180003C2400003C2400003C2400003C240000EF
:100190003C2400003C2400003C2400003C240000DF
:1001A0003C2400003C2400003C2400003C240000CF
:1001B0003C2400003C2400003C2400003C240000BF
:1001C0003C2400003C2400003C2400003C240000AF
:1001D0003C2400003C2400003C2400003C2400009F
:1001E0003C2400003C2400003C2400003C2400008F
:1001F0003C2400003C2400003C2400003C2400007F
:10020000B4280000000000008344550050000000A6
:1002100000277800000006000A0000008444520015
:100220004F5000003E007800000006000A00000069
:1002300084535700414200000080FD00000006008A
:100240000A000000834E4900500000000E87E800BD
:10025000000006000A000000C4545500434B000093
:100260001E27780010079800000006000C00000010
:10027000C4535700415000009E1F7800000F7800C3
:100280004F007800000006000E000000C44F56002A
:1002900045520000002778001E0090000000060074
:1002A0000C000000C3524F0054000000801F780073
:1002B0001E0090003E0F78004F27780000000600D7
:1002C00010000000C4504900434B00000000E9004A
:1002D000000040006E007800000006000E000000E4
:1002E000C4504F004B4500000000E90000004000F2
:1002F0000E0040003E0878003E0078000000060036
:1003000012000000C4524F004C4C00000000E900F5
:100310000C003400811F7800821F78008E0040009E
:1003200081004000911F7800010178000000E90081
:1003300000800900C21078004F0F78004F0178004C
:10034000CF0078003E007800000006002600000084
:10035000C43F4400555000000000B00001003200CE
:1003600000277800000006000E000000823E5200C8
:10037000801F78003E007800000006000A000000A0
:1003800082523E00002778004F00780000000600EF
:100390000A00000082524000002778007FB89700D2
:1003A000000006000A0000008140000010007800F4
:1003B0000000060008000000C24340001040780022
:1003C0000000FB00000006000A000000C121000040
:1003D0003E0878003E007800000006000A00000099
:1003E000C24321001E4878003E0078003E0078009D
:1003F000000006000C000000812B00003E004000C1
:100400000000060008000000C22B2B00811F7800AE
:10041000BE0078003E0040001E8F4800CF007800EC
:100420000000060010000000864E450047415400C1
:10043000450000000000EA00000006000C0000007B
:10044000812D00003E0010000000060008000000A2
:10045000C22D2D00811F7800BE0078003E001000E4
:100460001E8F1800CF00780000000600100000006A
:1004700082322A004100DD00000006000800000072
:1004800082342A004200DD0000000600080000005F
:1004900082322F004180DE000000060008000000CC
:1004A00082342F004280DE000000060008000000B9
:1004B00082303C004F80DE00000006000800000093
:1004C000C2303D000000B000010032000080EF00AB
:1004D0000080EA00000006000E000000C2303E006E
:1004E0000000B000020032000080EA004F80DE0011
:1004F000000006000E000000C2553C003E00100047
:100500000000EF00F2FF3900000006000C000000C0
:10051000C13C00003E0010000000EF00ECFF350081
:10052000000006000C000000C13D00003E00680015
:100530000000EF00E6FF3200000006000C000000A3
:10054000C13E00003E0010000000EF00E0FF3C0054
:10055000000006000C000000C34E4F0054000000D5
:100560000000B000DAFF32000000EF0000000600DB
:100570000E000000C2552A00811F78003E00B8001E
:10058000CF007800000006000C000000C12A000027
:10059000811F78003E80B900CF007800000006007F
:1005A0000C000000C5552F004D4F4400821F7800FD
:1005B000811F7800000178001E00780011000900FA
:1005C0000280D800010F7800CF0078004F0178003A
:1005D000000006001A000000C6552A002F4D4F00EB
:1005E00044000000821F7800811F7800000178001D
:1005F0003E0078001E00B800110009004288D800B3
:10060000010F7800CF0078004F017800000006004D
:100610001E000000C52A2F004D4F4400821F7800A5
:10062000811F7800000178003E0078001E80B9002C
:10063000110009004208D800010F7800CF007800AF
:100640004F017800000006001C000000C42F4D0080
:100650004F440000821F7800811F7800000178005D
:100660001E007800110009000200D800010F780078
:10067000CF0078004F017800000006001A0000004B
:10068000C12F0000811F780080007800F1FF070073
:1006900001F0A300010039008100EA00801F78000A
:1006A0003E00780000F0A300010039000000EA00DD
:1006B0004100DD00810050004F007800CF0078003D
:1006C0000500390000F0A300020031000000E8003E
:1006D000000006000000E9000000060030000000F5
:1006E000C34D4F0044000000DAFF07003E007800D1
:1006F000000006000C000000C22A2F00811F7800B5
:1007000080007800C5FF0700E1FF37000000060009
:100710000E000000C453510052540000831F7800A3
:10072000821F7800811F78000027EB00010820005D
:100730001E8140000211B8000200E10001003900F2
:100740001E8F40008100D100F9FF39001E01E80032
:100750001E11B8000010E100010031001E0FE8007A
:10076000CF0078004F017800CF0178003E0078007C
:100770000000060032000000C34D41005800000098
:100780001E00E10002003C003E0078000000060070
:10079000620747000000060012000000C34D490038
:1007A0004E0000001E00E100F9FF35003E00780019
:1007B000000006000E000000C3414200530000008C
:1007C0000000B00001003B000000EA00000006004D
:1007D0000E00000083414E00440000003E00600017
:1007E000000006000A000000824F52003E00700028
:1007F000000006000800000083584F00520000006F
:100800003E006800000006000A000000C3415300DB
:10081000480000000000B0000800320004003B0067
:100820000080EA00008009001E8FD100030037001D
:100830000000E900008009001E0FD0003E00780093
:10084000000006001E000000C34C530048000000DA
:100850000000B000F9FF3200F5FF3B000080EA0025
:10086000008009001E0FD100F4FF370000000600D1
:1008700016000000C3524F004C0000000000B00002
:10088000EEFF320004003B000080EA000080090017
:100890001E0FD300E9FF37000000E90000800900C7
:1008A0001E0FD200E5FF3700000006001E0000000A
:1008B00083434F004D0000000080EA000000060066
:1008C0000A000000C32B430021000000811F7800B4
:1008D000BE00780010C840003E007800CF007800CD
:1008E0000000060012000000C32D4300210000009C
:1008F000811F7800BE00780010C810003E0078000C
:10090000CF0078000000060012000000C22B21007A
:10091000811F7800BE007800108840003E007800FB
:10092000CF0078000000060010000000C22D21005A
:10093000811F7800BE007800108810003E0078000B
:10094000CF0078000000060010000000C4464900F7
:100950004C4C0000821F7800811F78003E01780017
:10096000BE0078000201E90002800900805878008A
:100970003E007800CF0078004F01780000000600AC
:100980001C000000C5434D004F564500821F7800F3
:10099000811F78003E0178009E001100BE007800A3
:1009A000050039000000E90009003300008009005B
:1009B00031597800060037000201400081004000F4
:1009C0000000E90002003300008009004161780066
:1009D0003E007800CF0078004F017800000006004C
:1009E00030000000C44D4F0056450000821F7800C3
:1009F000811F78003E0178009E001100BE00780043
:100A0000050039000000E9000B00330000800900F8
:100A1000311978000800370002014000020140004F
:100A200081004000810040000000E9000200330026
:100A300000800900412178003E007800CF00780056
:100A40004F01780000000600340000008449440093
:100A50004C4500000140FE00000006000A000000B6
:100A600085534C00454550000040FE000000060044
:100A70000A000000C8535F0054414D00504F4E0023
:100A80000027780000802000000006000E00000013
:100A9000C6535F00574F5200440000000027780003
:100AA00000862000000006000E000000C8535F0012
:100AB000464F52004D41540000277800008A200024
:100AC000000006000E000000C549540052583100D5
:100AD0000027780000902000000006000C000000B5
:100AE000C55445004C454300002778004090200045
:100AF000000006000C000000C6434E00544954009C
:100B000050000000002778006090200000000600E0
:100B10000E000000C3504100440000000027780090
:100B200020912000000006000C000000C33E490098
:100B30004E000000002778004091200000000600D1
:100B40000C000000C94D45004D5F44004550540065
:100B50004800000000277800609120000000060097
:100B600010000000CB4D45004D5F5000524748003B
:100B700045524500002778008091200000000600C3
:100B800010000000CA414400525F4300524541003A
:100B90005445000000277800C091200000000600A6
:100BA00010000000C5535400415254000027780043
:100BB00000922000000006000C000000C554450013
:100BC0004D5053000027780040922000000006009E
:100BD0000C000000C5544100434845000027780040
:100BE00060922000000006000C000000C84D450087
:100BF0004D5F480045524500002778008092200054
:100C0000000006000E000000CA5354004F505F0061
:100C1000464F52005448000000277800A092200060
:100C20000000060010000000C4454F004C4E0000BC
:100C300000277800E0922000000006000C00000071
:100C4000C3454F00460000000027780000932000B5
:100C5000000006000C000000C442410053450000A3
:100C60000027780020932000000006000C00000000
:100C7000C55354004154450000277800409320009C
:100C8000000006000C000000C5455200524F520003
:100C90000027780060932000000006000C00000090
:100CA000C9545F005355530050454E0044000000A6
:100CB00000277800C093200000000600100000000C
:100CC000C8505200494F520049544500002778004F
:100CD000E0932000000006000E000000CA494E000C
:100CE000505554005F4649004C45000000277800ED
:100CF000009420000000060010000000C7505200C1
:100D0000475F50004E54000000277800409F2000AD
:100D1000000006000E000000C54445005054480085
:100D200000277800E0DF20000E0050004180DE0048
:100D30000000060010000000C65244004550540058
:100D4000480000000027780040D0200000805700B5
:100D50004180DE000000060012000000C750520073
:100D6000474845005245000082FF070000277800F1
:100D7000801F78003E0078002000B000100078004E
:100D8000002778004F00780010007800000006006F
:100D90001C000000C83E5000524748004552450024
:100DA00074FF070000277800801F78003E0078005D
:100DB00087FD0700002778004F0078002000B00072
:100DC00083FD0700000006001C000000C4454D0024
:100DD00049540000002778000027780030012000E7
:100DE000D2FD07002BFD070000277800100120002E
:100DF000CEFD07003E007000D9FD07000000B000E6
:100E00003E0078001E00320037FF07001000780017
:100E10000000B0003E0078000E003200002778008D
:100E200080BB200030FF070069FD07000027780025
:100E3000A0002000BDFD07000000B0003E007800CB
:100E40000300320000277800E00220000100370094
:100E500000000600002778000000B0003E00780087
:100E600007003200A1FF07002008B00053FD070073
:100E700094FD07000000B0003E007800F9FF32004A
:100E8000002778000000280090FF07000027780066
:100E9000801F78003E00780000277800100078005E
:100EA000801F78003E00780049FD07000027780089
:100EB0002022200010007800002778000020200069
:100EC0003E0060000000B0003E00780003003200E9
:100ED0000027780000002000050037000027780078
:100EE000402220003AFD070000277800F0FF2F0085
:100EF0000000B0003E007800ECFF320000277800D0
:100F00004F007800002778004F00780030FD070080
:100F100000000600A6000000C45052004740000038
:100F200079FF0700811F7800821F7800BE007800DB
:100F30001000A7001500370002FC2F00028160009E
:100F40001010E10011003A00100190001E10E100A5
:100F50000E003A004000B000E103B2000080400003
:100F6000C108DE00008040000001EB000000A60088
:100F7000B0007800304178000000A600B000780092
:100F8000020F7800010078000500370022032000DE
:100F90001E0978001181BA00020F78001100BA0012
:100FA0004F017800CF007800000006004C000000E0
:100FB000C45052004721000053FF0700811F7800F2
:100FC000821F7800BE00780002FC2F0002816000C2
:100FD0001010E10003003A00100190001E10E10023
:100FE000060032001000A6002800070002FC2F00B7
:100FF000029860001E107800110007004000B00049
:10100000E103B20000804000C108DE000080400023
:1010100062074700BE0078003E0178000000A6008D
:1010200001187800025878000000A6000118780026
:101030003E0078004F017800CF00780000000600E5
:10104000811F7800821F7800831F7800841F78003A
:10105000B00078002203200030097800F30020005F
:101060001101BA003182BA000218780004587800E1
:101070001101BA003182BA000458780002187800D1
:101080008301E900F6FF31002A003700811F780054
:10109000821F7800831F7800841F780021042000BD
:1010A000020E2000911F780091087100B0007800B6
:1010B00082052400023B88002203200030097800CA
:1010C0008108BB0052052000323B8800A20A2000A4
:1010D000323B880061E7A80000000000000000002B
:1010E00042002400023B8800F30020003001780019
:1010F000304278008208BB008498BB003042780000
:10110000300178008208BB008498BB008301E900AD
:10111000F6FF310052052000323B8800A20A200071
:10112000323B880061E7A8000000000000000000DA
:101130004200F9004006B1004F027800CF0178006C
:101140004F017800CF00780000000600D0000000BA
:10115000C4505200472C000003FF07004DFC07005D
:101160004CFC0700002778000000200000277800D2
:1011700020002000A5FC070009FF07008EFF0700E4
:10118000000006001C000000C4454500504000005F
:10119000811F780021032000BE0878001000BA00EB
:1011A000CF0078000000060012000000C445450092
:1011B00050210000811F7800821F780082052400E2
:1011C000023B880021032000BE0878000001EB00EC
:1011D0000208BB000500FC0052052000323B8800DD
:1011E000A20A2000323B880061E7A800000000004E
:1011F0000000000061E7AF00FEFF3700420024005E
:10120000023B88003E08BB000500FC0052052000A0
:10121000323B8800A20A2000323B880061E7A80028
:10122000000000000000000061E7AF00FEFF370093
:101230003E0078004F017800CF00780000000600E3
:101240004C000000CB7370005F7379006E63700018
:1012500072672100ACFE07001000A6008BFF07009C
:101260001000A0003E0078000000060062000000B0
:10127000C4484500524500005FFE0700100078009A
:10128000000006000C000000C53E48004552450025
:1012900059FE07004EFC0700000006000C0000008D
:1012A000C2432C00F4FF0700002778001000B000B4
:1012B000F7FF07004BFC07000000060010000000CD
:1012C000C12C0000ECFF0700002778002000B000D0
:1012D000EFFF07003EFC07000000060010000000C2
:1012E000CA7370005F636F006D7069006C65000009
:1012F000E8FB0700E7FB070009FF0700801F7800F5
:101300003E007800002778003E0068000027780043
:101310007FB8970000277800F00320003E006000AF
:101320001000B0000027780030002000C9FC070042
:10133000D1FB07006AFC07003E0010004100DD0001
:1013400032FC0700002778004F0078000027780063
:10135000000420003E0060000000B0003E00780065
:101360003100320080FE07000027780000002000D6
:10137000002778002000200024FC070035FC07002F
:10138000C4FB070000277800F0FF2F0067FC070070
:101390000000B0003E0078000D003200801F780091
:1013A0003E0078003E0078000027780070002000A2
:1013B000002778004F0078004180DE000027780089
:1013C000000028003E00700063FF07001500370092
:1013D00065FE070000277800000020000027780045
:1013E0002000200009FC070008FC0700801F78008F
:1013F0003E007800002778002000200000277800B9
:101400004F00780054FF0700801F78003E007800EE
:101410000027780000002000002778004F007800A7
:101420004DFF0700170037009AFB070099FB0700E4
:10143000BBFE070048FF07000027780000002000DF
:101440000027780020002000F0FB070091FB070038
:1014500090FB0700B2FE07001AFC070086FB07009E
:10146000002778006000200030FC07003E0060008C
:101470000000B0003E007800EBFF32003E00780034
:101480003E00780000000600E600000042494600E9
:1014900000277800000B20000027780000002000C3
:1014A0002DFF070000277800800720000027780024
:1014B000E003200028FF0700002778002003200019
:1014C00000277800F0FF2F0023FF070026FE07000B
:1014D0000000060026000000C77370005F73610003
:1014E00075740000801F78003E007800801F78002F
:1014F0003E00780067FB070066FB070000277800C6
:10150000000020000027780020002000D1FB070009
:1015100083FE07003E007800002778004F00780027
:10152000002778004F007800002778005000200046
:1015300066FB0700002778005000200063FB0700CF
:10154000C4FB0700801F78003E0078000027780069
:10155000F0002000BEFC0700002778004F00780054
:1015600000277800F0FF2F00B9FC07003E00400084
:10157000002778004000200064FB07000027780067
:101580004000200061FB07000027780000002000D9
:101590000027780020002000AEFB070086FE070031
:1015A000000006008E00000044454C00534500003A
:1015B000002778007003200000277800F0FF2F003C
:1015C000E5FE0700E8FD0700C6FF0700E6FD07008F
:1015D000000006001800000044544800454E00007A
:1015E000E1FD0700BFFF0700000006000C0000003F
:1015F00044434100534500000027780000002000CC
:1016000000277800002778000000200000277800DD
:10161000601B200036FF07000000060018000000D5
:10162000424F460000277800000020000027780085
:10163000A01C20002EFF07000027780000002000DB
:10164000002778004029200029FF070090FF0700AD
:10165000000006001C00000045454E00444F4600B7
:10166000D3FF0700000006000A00000047454E00B7
:101670004443410053450000A9FD07004180DE00BE
:1016800035FB07000000B0003E0078002500320066
:1016900000277800300020000CFB070000277800AE
:1016A0003000200009FB07003E0070000000B00081
:1016B0003E00780008003200801F78003E0078006D
:1016C000A9FD070087FF0700002778004F0078007A
:1016D0001000B100020037003E0078003E007800A4
:1016E0000027780077FB07000000B0003E0078007C
:1016F000E7FF32003E00780000277800000020005D
:1017000000277800001C2000F9FE07000027780061
:101710000000200000277800E0102000F4FE070001
:101720000200370000277800F0FF2F0000000600BD
:10173000640000004542450047494E008AFD07000D
:10174000000006000A00000045554E0054494C00B8
:101750004FFF07000027780040002000EBFA070049
:101760000027780040002000E8FA07005DFF07002E
:10177000000006001800000045574800494C45008D
:1017800043FF0700000006000A0000004652450023
:10179000504541005400000085FF070000277800F5
:1017A00040002000D9FA0700002778004000200000
:1017B000D6FA07004BFF0700000006001A000000E1
:1017C00042444F00002778000000200000277800E6
:1017D00080132000C6FE070063FD07000027780085
:1017E0000000200000277800601B2000C0FE0700DA
:1017F000002778000000200000277800601B2000F0
:10180000BBFE07000000060026000000452B4C0030
:101810004F4F50000027780000002000002778007C
:10182000001C2000B2FE0700002778000000200006
:1018300000277800C01F2000ADFE070000277800B9
:101840000000200000277800001C2000A8FE0700F0
:101850000027780000002000002778006014200096
:10186000A3FE070000277800000020000027780072
:10187000601420009EFE0700002778000000200072
:10188000002778008028200099FE070000277800B4
:101890000000200000277800C02A200094FE0700E6
:1018A000ABFF070000277800000020000027780029
:1018B000E01020008EFE07000027780000002000C6
:1018C00000277800E010200089FE070000000600D5
:1018D00064000000C74C490054455200414C0000D0
:1018E0000027780080072000002778000070220081
:1018F00019FE070000277800801F78003E0078005E
:101900000027780040FF2F00D1FB07000002B00045
:10191000002778004F007800002778004000200062
:10192000CBFB07000CFE07004AFE07000000060084
:1019300030000000444C4F004F500000002778005A
:1019400010002000E6FF0700B2FF070000000600BD
:101950001000000081490000002778007FB8970040
:10196000000006000A000000814A000000277800FD
:101970005FB89700000006000A000000814B0000DD
:10198000002778003FB89700000006000A0000001A
:10199000854C450041564500002778004F007800EF
:1019A0004F007800801F7800801F78003E0078008C
:1019B000000006001400000084455800495400004F
:1019C0000000060008000000C24352000027780013
:1019D000D0002000FFFC070000277800A0002000B6
:1019E000FCFC07000000060012000000C442450095
:1019F0004C4C00000027780070002000F5FC070028
:101A0000000006000E000000C55350004143450091
:101A10000027780000022000EEFC0700000006000E
:101A20000E000000C6535000414345005300000023
:101A300049FA07000000B0003E00780008003200BC
:101A4000F3FF07001000B100002778009DFA07009F
:101A50000000B0003E007800F9FF32003E00780040
:101A60000000060022000000C45459005045000048
:101A7000002778009AFA07000000B0003E007800C6
:101A80002F0032001000B100801F78003E00780067
:101A90000027780049FA070000277800F00F20009F
:101AA0003E0060000027780086FA0700F9F9070079
:101AB00000277800300020009CFA07003E007000EC
:101AC0000000B0003E007800090032003E007800BF
:101AD000002778004F0078003E007800002778004B
:101AE00000002000801F78003E0078000B003700C7
:101AF0000027780000277800D00020008BFA07002C
:101B00000000B0003E007800030032003E00780084
:101B1000AEFF070001003700AEFC07001000B00068
:101B2000002778004F0078000027780065FA07004A
:101B30000000B0003E007800D2FF3200690037009C
:101B4000002778004F80DE000000B0003E007800E3
:101B500064003200801F78003E007800CDF9070055
:101B6000CCF90700EEFC0700002778004F00780052
:101B70000000EA00002778000000B0003E00780076
:101B800014003200801F78003E00780000277800A3
:101B900080FF2F002EFB0700002778000027780029
:101BA000D000200061FA07000000B0003E0078007D
:101BB000030032003E00780084FF07000100370078
:101BC00084FC0700002778004F0078001000B10067
:101BD00002003700A8F907003E00780000277800CF
:101BE000801F78003E0078000000B0003E007800C2
:101BF000110032000027780000277800D000200074
:101C00004AFA07000000B0003E00780003003200EE
:101C10003E0078006DFF0700010037006DFC0700F3
:101C2000002778004F0078001000B100801F780076
:101C30003E007800010037003E0078000027780061
:101C4000000020000027780020002000EFF90700A6
:101C500090F907008FF90700B1FC07000027780012
:101C60004F007800002778000000B0003E007800A8
:101C700014003200801F78003E00780000277800B2
:101C800000277800F00F20003E0060000027780059
:101C900000277800D000200024FA07000000B000E0
:101CA0003E007800030032003E00780047FF070046
:101CB0000100370047FC0700002778004F0078003C
:101CC0001000B10000277800FEF907000000B00006
:101CD0003E007800A7FF32003E0078003E0078000A
:101CE0003E0078003E0078003E00780000000600CC
:101CF00046010000C5434F00554E540000277800B0
:101D00001000B0005CF90700ACF90700002778006C
:101D1000F00F20003E0060000000060016000000EA
:101D2000C92D5400524149004C494E004700000063
:101D300000277800EAF9070000277800300020002B
:101D400062F9070000277800300020005FF90700E3
:101D50001000B1003E00400098F90700002778000D
:101D600000022000F1F907003E0060000000B00012
:101D70003E007800020032001000B100ECFF370096
:101D80000000060034000000C34249004E0000007D
:101D90000027780020002000B1FB07008CF9070025
:101DA0000000060010000000C54F430054414C00E5
:101DB0000027780080002000A9FB070084F90700B5
:101DC0000000060010000000C744450043494D00D4
:101DD000414C000000277800A0002000A0FB070075
:101DE0007BF907000000060012000000C348450010
:101DF00058000000002778000001200098FB070031
:101E000073F907000000060010000000C7434F00F0
:101E10004E564500525400001000B00000277800D4
:101E2000000020001BF9070064F907000027780074
:101E300000277800B0022000BCF907000000B000C5
:101E40003E007800070032003E007800801F7800D6
:101E50003E0078001000B000002778004F007800A6
:101E60000C00370000277800D0022000AFF90700EF
:101E70000000B0003E00780006003200801F7800AD
:101E80003E0078001000B000002778004F00780076
:101E90001000B100801F78003E0078000027780015
:101EA00046F907000003B100002778004F80DE00EC
:101EB0000000B0003E007800040032003E007800D0
:101EC00000277800F0FF2F0035003700002778004A
:101ED00000277800900020009AF907000000B00069
:101EE0003E007800060032007000B1000027780044
:101EF00000277800A000200086F9070002003700C4
:101F000000277800000020000000B0003E007800AC
:101F1000040032003E00780000277800F0FF2F0018
:101F20001F003700002778004DFB070010007800E5
:101F300078F907000000B0003E007800150032007C
:101F4000801F78003E007800801F78003E007800F7
:101F500043FB07001000780087F90700002778008E
:101F60004F0078001000B000002778004F00780084
:101F7000C1F80700801F78003E0078003E00400056
:101F8000002778004F00780000277800000020002C
:101F9000030037003E00780000277800F0FF2F0094
:101FA0000000B0003E007800BCFF3200002778003F
:101FB0004F0078000000B0003E00780005003200BD
:101FC000801F78003E0078000000EA0000277800BB
:101FD0004F00780000000600E8000000C23C23002B
:101FE0000027780000002000B3FA0700FDF8070082
:101FF00000277800801F78003E0078004F80DE00C8
:10200000002778004F007800EDF907000000060077
:102010001C000000C4484F004C440000A6FA070012
:10202000002778001000B000002778001000B000F2
:102030000027780030002000A4F80700DFF8070030
:1020400000277800F00F20003E0060000027780095
:10205000E0052000D3F907004CFA070000277800BC
:10206000D6F8070000277800F00F20003E0060003F
:102070001000B00000277800E0052000C9F9070033
:1020800084F80700D7F807001000B000D5F8070063
:102090000000060042000000C1230000F0FA070023
:1020A0001000780041F9070073F807000003B00042
:1020B00000277800002778009003200021F907000E
:1020C00000277800700020003E0060003E004000C5
:1020D000D2FF07000000060022000000C2235300C8
:1020E000EEFF0700002778001DF907000000B00090
:1020F0003E007800FAFF32000000060012000000E7
:10210000C4534900474E000062F807000000B000C9
:102110003E0078000300320000277800D002200043
:10212000BEFF07000000060016000000C2233E00AC
:102130003E0078003E0078005FFA0700EFFE0700DF
:10214000000006000E000000C12E0000A4FF0700E2
:102150000027780000022000B0FF0700E0FF070022
:10216000E9FF0700F2FF070041FE0700000006003C
:1021700016000000C13F000010007800F3FF0700C8
:10218000000006000A000000C2552E00002778005B
:102190000000200092FF07000027780000022000C6
:1021A0009EFF07003E00780033F80700CCFF0700D1
:1021B000DFFF07002EFE0700000006001C000000E5
:1021C000C4574F0052440000801F78003E00780042
:1021D00032FA070000277800000020002DF80700E1
:1021E00080F80700002778000000200090FA070020
:1021F00077F80700002778000000200092FA070017
:1022000073F8070045FA07001000780049FA070044
:10221000100078003E00400000277800801F780002
:102220003E0078001000B000002778001000200069
:1022300040FA0700B6F90700002778004F00780041
:102240005EF8070000277800F00F20003E006000D5
:1022500000277800801F78003E0078000027780073
:102260003000200019F807000027780053F8070015
:102270003E0040001000B0005AF807000027780028
:102280004F007800002778008EF8070001F807005B
:102290000027780030002000A4F807003E007000FE
:1022A0000000B0003E0078000A0032003E007800D6
:1022B00000277800F0FF2F00002778005CFA070065
:1022C00043F80700002778005FFA070040F807008E
:1022D0002E0037000027780000277800D00020006B
:1022E00092F807000000B0003E00780007003200BE
:1022F0003E00780000277800F0FF2F0000277800CC
:102300004BFA070032F8070020003700002778005A
:10231000801F78003E0078000027780090002000A1
:1023200082F80700002778007FB897000027780020
:10233000000220007DF807003E00700000277800B2
:102340004F007800002778007FB8970077F80700E3
:102350003E0070000000B0003E0078000300320034
:1023600000277800F0FF2F000800370000277800D2
:10237000100020000027780030002000D3F707006D
:1023800052F9070000277800000020000000B0008C
:102390003E007800A0FF32003E0078000027780061
:1023A0004F0078003E00780000000600F8000000B2
:1023B000C1270000002778000002200082FF0700EC
:1023C00000277800FDF707000000B0003E0078000D
:1023D000CE003200801F78003E007800F3F907003D
:1023E00000277800801F78003E0078002000B000B1
:1023F00010007800002778004F0078001000780067
:10240000002778007FB89700002778000027780021
:10241000EAF707003E0040001000B00000277800F7
:1024200040002000A9F707000027780040002000A6
:10243000A6F7070097F7070096F70700B8FA070016
:1024400000277800F0F32F003E006000002778009E
:102450004F0078008FF7070000277800F00F20006A
:102460003E0060008BF70700D4F7070000277800D4
:10247000F00F20003E0060002CF807000000B000C4
:102480003E007800350032001000B00000277800D0
:10249000600020008DF707007EF7070029F807008D
:1024A0000000B0003E0078002900320079F70700F4
:1024B0000027780080FF2F00E5F8070075F7070078
:1024C000BEF7070019F807000000B0003E007800D2
:1024D0001C0032001000B0000027780060002000CF
:1024E0007AF707006BF7070016F807000000B00046
:1024F0003E007800100032000027780030002000F5
:1025000072F7070063F70700ACF7070007F807004A
:102510000000B0003E007800040032001000B0005F
:1025200000277800F0FF2F00020037000027780016
:10253000000020000200370000277800F0FF2F0085
:10254000020037000027780000002000020037005A
:1025500000277800F0FF2F000200370000277800E6
:1025600000002000801F78003E007800801F780067
:102570003E0078003E0078003E007800002778009A
:102580004F007800002778004F0078000000B0006E
:102590003E0078001F003200002778004000200035
:1025A0004AF707003BF70700E6F707000000B00016
:1025B0003E0078000F003200801F78003E00780057
:1025C000002778000000200000277800200020006D
:1025D0008EF707002FF707002EF7070050FA0700C5
:1025E000002778004F0078000027780000002000C6
:1025F000070037003E0078003E0078003E0078007B
:102600003E0078003E00780000277800F0FF2F00A1
:102610003A0037003E0078003E0078003E00780027
:10262000801F78003E007800801F78003E00780010
:1026300018F7070017F707000027780000002000B0
:10264000002778002000200082F7070034FA0700F6
:1026500010F707000FF707003E0070000000B00001
:102660003E007800170032007AF707000027780054
:102670004F007800002778004F007800002778008E
:102680004000200011F707000027780040002000DC
:102690000EF70700FFF60700FEF6070020FA070016
:1026A00000277800F0F32F003E006000002778003C
:1026B0006000200005F707000027780000002000D8
:1026C0000E003700002778004F00780000277800C0
:1026D0004F0078003E0078003E0078003E00780011
:1026E0003E0078003E007800002778003E00680039
:1026F0000027780000277800F0FF2F000000B000CE
:102700003E00780053FF32000300370000277800B6
:102710003E0068000027780000000600B8010000B5
:10272000C44649004E44000022FF0700D9F60700C6
:10273000D8F607003E0070000000B0003E007800B0
:1027400015003200D3F60700D2F60700F4F90700AF
:10275000801F78003E007800002778003E00680067
:10276000002778004F00780000277800F003200051
:102770003E0060001000B00000277800300020000C
:10278000B4F70700BCF6070055F707003E0010003D
:102790004100DD001DF707000000060040000000BA
:1027A000415B0000002778000000200032F907009C
:1027B00007F70700000006000E000000C15D0000E2
:1027C00000277800F0FF2F002BF9070000F7070023
:1027D000000006000E000000C13A0000002778004B
:1027E0000002200078FE07005FF90700002778004C
:1027F00000002000002778002000200003F70700D9
:10280000EAF8070000277800801F78003E00780073
:102810002000B00010007800002778007FB89700F3
:10282000100078000BF707004BFA07004EF907007D
:10283000002778007FB89700E5F6070000277800AA
:102840004F0078002000B000E1F607000027780074
:10285000DAF6070000277800F00320003E00600051
:102860001000B000801F78003E007800002778003C
:102870002000B000D1F6070000277800F00F2000FC
:102880003E00600083F607001000B000CBF60700A2
:102890000027780080002000EDF70700002778006F
:1028A0007FB897001000B10000277800000C2000CE
:1028B0003E0070003E00400027FA07003000B000E4
:1028C000002778004F0078003000B1000027780022
:1028D00003F707000000B0003E0078001600320049
:1028E000801F78003E007800002778002000B000AC
:1028F000B2F6070000277800F00F20003E006000CD
:1029000064F607001000B000ACF60700002778005E
:1029100080002000CEF7070000277800300020005C
:102920006AF60700A5F6070000277800F00F2000E0
:102930003E006000DFFF37003E0078003E00780078
:1029400000277800F0FF2F00CBF80700A0F6070063
:10295000F3F807007FF807009DF607000000060067
:10296000C6000000413B0000002778006000200006
:102970000027780000002000F7F9070035FA07006B
:102980000027780000002000BBF8070090F6070041
:10299000E3F807006FF80700100078003E00100011
:1029A0000000B0003E0078000E00320000277800E2
:1029B00030002000B6F8070085F6070057F807003A
:1029C00010007800B2F807002000B00080F6070081
:1029D00058F8070010007800ADF807004000B0007C
:1029E0007BF607000000060044000000C87370007A
:1029F0005F74610063686500002778004F0078000D
:102A0000002778004F007800002778003000200071
:102A10002EF6070000277800801F78003E0078001F
:102A20008000B0006AF60700002778004F007800A9
:102A3000A000B00066F60700000006006E0000006F
:102A4000C6544100434845003A00000063FF0700B8
:102A500009FA0700A2FB0700002778000000200009
:102A600018FA0700002778000000200015FA070078
:102A7000002778000000200012FA070000277800E5
:102A8000000020000FFA0700002778000000200057
:102A90000CFA0700002778000000200009FA070060
:102AA000002778000000200000277800604F2100F8
:102AB0000FFA0700000006003E000000C9545F0046
:102AC0004558450043555400450000000027780054
:102AD000801F78003E007800A000B0001000780051
:102AE000002778004F0078008000B00010007800C8
:102AF000801F78003E007800801F78003E0078003C
:102B00000000060026000000C8545F00414A4F0044
:102B10005554450066F8070000277800801F7800AC
:102B20003E0078001000780000277800F0FF2F00AA
:102B3000002778007FB8970025F60700801F7800EF
:102B40003E00780025F80700002778001000780084
:102B500001F607000000B0003E00780035003200AA
:102B60000027780030002000D8F50700C9F50700DD
:102B70006EF607000000B0003E007800070032004B
:102B80003E0078003E0078003E0078003E0078006D
:102B900000277800F0FF2F0025003700002778007D
:102BA000100078000027780050002000C7F50700CB
:102BB00052F607000000B0003E007800140032001A
:102BC0000027780030002000C0F507004000B0006A
:102BD000FFF50700801F78003E007800002778008E
:102BE000002778004F007800F9F5070000277800EB
:102BF000F0FF2F00A7F507002000B000F4F5070054
:102C0000F3F5070000277800F0FF2F0008003700D9
:102C1000801F78003E0078003E0078000027780092
:102C20004F0078004000B00000277800000020002E
:102C300013003700801F78003E00780000277800DE
:102C4000002778004F007800E1F5070000277800A2
:102C5000F0FF2F008FF507002000B000DCF5070023
:102C600000277800000020008AF507004000B0002F
:102C7000D7F50700D6F5070000277800F0FF2F00F2
:102C80000000B0003E007800AFFF3200002778005F
:102C90004F007800002778004F007800CCF507003F
:102CA00000000600D0000000C8545F0041435400FB
:102CB00049564500801F78003E00780000277800C4
:102CC00010002000AEF60700002778000000220068
:102CD000B4F60700002778004F0078006000B000CD
:102CE000BBF507000000060022000000C9545F0089
:102CF00050455200494F440045000000801F7800B5
:102D00003E00780000277800100020009CF60700A5
:102D10000027780000002200A2F6070000277800B4
:102D20000000EA00002778007FB897006000B0003C
:102D3000A7F507004180DE00A2F707001000780029
:102D40003E00400000277800F0FF27003E006000B2
:102D5000002778004F0078002000B0009CF50700A5
:102D6000000006003E000000C8545F0052455400B9
:102D70004952450078F507000000B0003E00780099
:102D80003D003200CAF7070000277800801F780056
:102D90003E0078001000780000277800F0FF2F0038
:102DA000002778007FB8970089F50700801F78001A
:102DB0003E00780089F7070036F5070035F5070073
:102DC00010007800D9F507000000B0003E00780040
:102DD00015003200801F78003E0078000027780040
:102DE000000020002BF507006000B00078F5070018
:102DF000002778004000B00010007800002778001D
:102E00004F00780072F507000027780000002000CE
:102E100020F507004000B0006DF50700002778009E
:102E2000F0FF2F000B003700100078004AF5070074
:102E30000000B0003E007800040032004000B00006
:102E400000277800000020000200370000277800EB
:102E5000F0FF2F000000B0003E007800D6FF3200E7
:102E60003E007800002778004F00780000277800A7
:102E70004F00780056F50700000006008C000000A7
:102E8000C57370005F2E6700002778004F00780040
:102E9000002778004F007800FEF40700FDF40700DB
:102EA0001FF8070000277800F00F20003E006000A8
:102EB000801F78003E0078003E007800F5F407009F
:102EC000F4F40700002778000000200000277800B5
:102ED0007FB897001000B000002778003000200075
:102EE000DCF50700E4F407007DF507003E00100064
:102EF0004100DD0045F50700002778004F0078000D
:102F0000DDF40700801F78003E007800DAF4070047
:102F1000801F78003E0078000000EA00D4FA070025
:102F200000000600E0000000C5544C004953540066
:102F30002AF707001000780007F507000000B0002E
:102F40003E0078007000320000277800A000B0003A
:102F500010007800CFF407008000B0001000780067
:102F600000277800000020000027780020002000C3
:102F700038F50700C7F40700C6F40700E8F70700B4
:102F80003E007800002778008007200067F50700E2
:102F90000000B0003E007800F1FF3200002778000A
:102FA00000002000002778002000200029F50700FD
:102FB000B8F40700B7F40700D9F70700801F7800BE
:102FC0003E0078003E007800002778004F0078002F
:102FD0000027780000277800000820003E006000ED
:102FE0000000B0003E0078000900320000277800A1
:102FF000F00320003E0060000000EA009CFA070099
:1030000083FA070000277800F0FF2F000200370046
:10301000002778003E0068000000B0003E00780005
:10302000DEFF32000EF7070010007800801F7800E6
:103030003E00780067FB070093FF07000B707200EB
:10304000696F720069746500203A200000277800DB
:10305000100078004DFC07002000B0000027780029
:103060004000B00010007800002778004F80DE009C
:103070000000B0003E0078000B00320082FF070025
:103080000D70650072696F006469710075652000DC
:103090003A2078000000EA002CFC07007AFF0700C5
:1030A000026D7300110037003E00780000277800A1
:1030B000100078004F80DE000000B0003E00780075
:1030C0000600320070FF070009494E0041435400DA
:1030D0004956450020652000040037006AFF0700BC
:1030E0000741430054495600452045000027780019
:1030F0004F007800DAF60700B5F4070033FA07004E
:103100002000B0008BFF370000000600F400000034
:1031100047434F004D5049004C450000A5FC0700B7
:103120005CF407005BF407003E0070000000B00094
:103130003E007800090032004FF40700E8F907006C
:10314000E7F907000027780000002000002778003A
:103150000097200066F80700100037003E00780056
:103160003E0078000027780030002000C8F60700F5
:1031700097F4070069F6070010007800C4F607000E
:103180002000B00092F407006AF6070010007800F3
:10319000BFF607004000B0008DF4070000000600F5
:1031A0004A000000495B43004F4D5000494C450028
:1031B0005D0000007FFC070036F4070035F40700CF
:1031C0003E0070000000B0003E00780002003200B7
:1031D00047F80700100037003E0078003E007800F6
:1031E0000027780030002000A9F6070078F40700D7
:1031F0004AF6070010007800A5F607002000B0008E
:1032000073F407004BF6070010007800A0F60700E3
:103210004000B0006EF40700000006003E00000011
:10322000C74558004543550054450000801F7800AD
:103230003E007800801F78003E0078000000060005
:1032400012000000C122000000277800400020008A
:1032500089F60700AEF50700C3F6070000277800DF
:10326000F00F20000027780000002000000006007A
:1032700018000000422E22000027780000002000E5
:10328000002778000074210019F80700EEFF0700FE
:10329000000006001200000001280000002778004E
:1032A0002000200074F6070099F5070000000600D2
:1032B0000E000000C22E530099F6070026F4070006
:1032C0000000B0003E0078001C00320000277800AB
:1032D00000002000801F78003E0078000027780062
:1032E0001000B000002778007FB897003E00100063
:1032F000F6F3070095FB0700002778004F007800E1
:103300001000B00000277800801F78003E00780091
:10331000E0F307007FF4070091F407000000B0001D
:103320003E007800EDFF3200002778004F00780063
:103330003E0078003E00780006003700D2FE07000D
:103340000C5069006C6520007669640065202100DE
:1033500020207800000006005400000049494D007C
:103360004D45440049415400450000000FF6070058
:1033700000277800801F78003E0078002000B00011
:1033800010007800002778004F00780010007800C7
:10339000C0F30700BFF30700E1F60700002778003D
:1033A000F0F72F003E00600000277800400020006A
:1033B000D6F307000027780040002000D3F3070071
:1033C000FDF60700000006003800000046444900F2
:1033D0005245430054000000F4F507000027780030
:1033E000801F78003E0078002000B00010007800B8
:1033F000002778004F00780010007800A5F3070040
:10340000A4F30700C6F6070000277800F0FB2F00A2
:103410003E0060000027780040002000BBF307005A
:103420000027780040002000B8F30700E2F607000C
:103430000000060036000000C5414C004C4F54000F
:10344000002778000000B0003E0078000500320040
:1034500000277800000020009AF707001000B10054
:10346000F7FF37003E007800000006001C00000057
:10347000C44C4F004144000005F6070010007800DE
:103480000000B0003E007800020032003E007800EC
:10349000F50137000DF6070010007800801F780056
:1034A0003E007800002778001000200007F6070093
:1034B000C7F3070099F5070010007800801F780017
:1034C0003E0078009BF5070010007800801F780010
:1034D0003E007800D6F5070010007800801F7800C5
:1034E0003E007800D8F5070010007800801F7800B3
:1034F0003E00780089F50700B5F307000027780043
:10350000000020008BF50700B1F30700DAF5070093
:103510001000780000277800F1F307000000B000E9
:103520003E007800B600320000277800200020001E
:1035300004F407000000B0003E007800A100320053
:1035400000277800200220001FFB0700EBF907008E
:1035500000277800300020005CF307000027780087
:10356000F00F2000E5F307004AF30700DCF3070043
:103570003E0060000000B0003E0078002C003200E9
:10358000801F78003E007800801F78003E007800A1
:1035900039F3070070F307000000B0003E00780028
:1035A0001700320000277800002778000010200064
:1035B000D2F307000000B0003E007800080032009F
:1035C000002778007FB897007CF307000027780079
:1035D000800020009EF407003E00400007003700F6
:1035E000002778007FB8970074F3070022F30700E4
:1035F000D9F60700002778000000200003003700FC
:10360000002778007FB897006CF307001AF30700D3
:103610001000B000002778004F0078001000B000C4
:10362000002778004F0078001000B100C8FF370075
:103630003E00780061F3070000277800002778003B
:1036400020022000B9F307000000B0003E0078001F
:103650002A0032003E007800801F78003E0078008B
:103660003DF307000000B0003E0078000400320087
:103670000027780000002000FFF20700B6F60700E0
:1036800004F3070003F3070025F60700002778007E
:1036900000F02F003E006000002778004F00780007
:1036A0003E004000002778004000200007F307009C
:1036B000002778004000200004F307003EF60700D2
:1036C0006DF507001000780000277800300020001A
:1036D00096F307000000B0003E00780002003200C0
:1036E0003E0078003E00780000277800400020006F
:1036F00061F507008EF407003100370052F507002E
:10370000100078000000B0003E0078000300320096
:103710003E00780000277800D0002000DDF207008E
:1037200000277800F00F200074F307000000B000BD
:103730003E00780021003200801F78003E007800B3
:10374000CDF2070004F307000000B0003E0078004F
:1037500015003200002778000027780000102000B4
:1037600066F307000000B0003E007800070032005A
:10377000002778004F0078000027780080002000A4
:1037800033F407003E0040000600370000277800B1
:103790004F007800B8F207006FF6070000277800A6
:1037A0000000200002003700002778004F0078005A
:1037B000B1F207001000B000010037003E007800B1
:1037C0000E00370000277800000220007EFA070074
:1037D00010007800002778001090220053F30700B3
:1037E0000000B0003E00780004003200002778009E
:1037F0002000200020F507004DF40700EB00370003
:103800003E007800EBFA0700A2F20700A1F20700E1
:103810003E0070000000B0003E0078005F00320003
:1038200015F50700100078000000B0003E00780099
:103830002400320097F2070096F20700B8F507005F
:103840008DF207003E007800002778000008200075
:103850003E0060000000B0003E0078000200320030
:10386000A3F60700160037008AF2070089F2070066
:10387000ABF50700801F78003E0078000027780035
:103880003E006800002778004F007800002778008D
:10389000F00320003E0060001000B0000027780018
:1038A000300020006BF3070073F207000CF30700F1
:1038B0003E0010004100DD00D4F207005BFE07006F
:1038C0003500370073F2070072F2070094F5070025
:1038D00069F207003E00780000277800000C200005
:1038E0003E00600000277800000420000FF307006E
:1038F0000000B0003E007800110032003E00780069
:103900003E0078000027780020002000E0F4070047
:10391000AFF2070081F4070010007800DCF4070024
:103920002000B000AAF2070082F40700100078001F
:10393000D7F407004000B000A5F2070016003700DA
:1039400054F2070053F2070075F50700801F780056
:103950003E007800002778003E00680000277800CD
:103960004F00780000277800F00320003E00600040
:103970001000B000002778003000200035F3070069
:103980003DF20700D6F207003E0010004100DD00C6
:103990009EF2070025FE0700840037003E007800F5
:1039A0003EF407000027780084F207000000B00012
:1039B0003E0078007B00320036F2070035F2070047
:1039C00015F9070039F207003E00780037F20700CA
:1039D0003E0078000027780078F207000027780082
:1039E00010022000CBF207000000B0003E0078007B
:1039F000080032003E0078009FF4070010007800B5
:103A00000000B0003E00780001003200B4F707006B
:103A1000630037000027780068F20700002778006D
:103A200000277800B0022000C0F2070012F2070061
:103A300000277800D0022000BCF207003E00700092
:103A400014F207001000B0005CF2070000277800B5
:103A500010022000AFF207003E0060000000B0003E
:103A60003E0078003E0032000AF207000000B0007D
:103A70003E0078003700320050F207007EF4070065
:103A8000100078000000B0003E00780027003200EF
:103A9000801F78003E00780000277800002778001B
:103AA0000040200095F207000000B0003E007800C2
:103AB0000E003200002778004000200064F3070069
:103AC000002778004F00780000277800D0022000FF
:103AD00096F2070000277800100020003E006000EA
:103AE000000BB000E4F107000E0037007CF7070080
:103AF0000027780000042000002778004F0078009D
:103B000000277800D002200088F207000027780004
:103B1000000320003E0060003E00100000277800F7
:103B2000E00320008CF5070009003700002778002B
:103B3000B00220007DF207000000B0003E007800D7
:103B4000020032003E004000010037003E0010003D
:103B5000020037003E0078003E0078001000370079
:103B60003E0078003E00780000277800100020001A
:103B700047F4070016F20700E8F30700100078008A
:103B800043F407002000B00011F20700E9F307003A
:103B9000100078003EF407004000B0000CF207006F
:103BA000020037003E0078003E00780026F407004F
:103BB0001000780036F40700100078003E00700016
:103BC0000000B0003E00780050FE320054F40700C0
:103BD0004F80DE000000B0003E0078000E00320092
:103BE000002778004000200029F40700F8F10700C2
:103BF000CAF307001000780025F407002000B00089
:103C0000F3F10700CBF307001000780020F4070061
:103C10004000B000EEF10700002778004F00780068
:103C200009F40700EAF10700002778004F00780048
:103C3000FFF30700E6F10700002778004F00780047
:103C4000BCF30700E2F10700002778004F0078007E
:103C5000B2F30700DEF10700002778004F0078007C
:103C60001AF40700DAF10700000006000004000063
:103C7000C643520045415400450000007EF5070050
:103C800017F7070038F40700C2F307000027780091
:103C9000801F78003E007800CDF1070000277800F3
:103CA0004F0078002000B000C9F10700002778001D
:103CB0004000200000277800F0FF2F0026F50700C5
:103CC000002778000000200000277800F00720007F
:103CD00021F507005FF5070000000600380000002E
:103CE000C87370005F646F0065733E00A9F307003E
:103CF00000277800801F78003E0078002000B00088
:103D000010007800002778004F007800100078003D
:103D10000027780000002000002778004F0078007E
:103D2000002778004000200068F107000027780095
:103D30004000200065F10700002778000000200007
:103D40000027780020002000B0F107009AF4070057
:103D50000027780040002000002778004F007800FE
:103D6000002778004000200068F107000027780055
:103D70004000200065F107008FF4070035F50700CB
:103D80000027780000002000BBF3070090F1070037
:103D9000000006009400000045444F0045533E00DB
:103DA00000277800000020000027780000E72100AD
:103DB0004FF507000000060012000000C856410041
:103DC00052494100424C450084FA0700ABFF07000E
:103DD0003CF50700C5FF07000000060012000000C8
:103DE000C8434F004E535400414E54007BFA070025
:103DF000BBF607000027780060002000002778004D
:103E000000002000D4F4070012F507000027780016
:103E10000000200098F307006DF107000000060085
:103E200022000000C653540052494E0047000000D3
:103E30006AFA070010F10700A9F60700A8F60700C4
:103E40000027780060002000002778000000200094
:103E5000C1F40700FFF407000027780000002000ED
:103E600085F307005AF10700000006002600000055
:103E7000C5564C00495354004CF307000027780006
:103E8000801F78003E0078002000B000100078000D
:103E9000002778004F00780010007800FDF0070040
:103EA000FCF00700FBF00700FAF007001CF4070025
:103EB000801F78003E0078003E00780000277800E0
:103EC0004F00780000277800F00320003E006000DB
:103ED0000000EA00E6F60700CDF60700EDF0070067
:103EE000ECF0070000277800000020000027780091
:103EF0002000200057F1070009F40700E5F0070053
:103F0000E4F007003E0070000000B0003E007800C2
:103F1000040032004FF10700002778000000200065
:103F2000040037003E0078003E007800002778004B
:103F3000F0FF2F000000B0003E007800D7FF3200F5
:103F40003E0078003E00780000000600700000008F
:103F5000C34B45005900000064F3070000277800B8
:103F60001000B00015F107000140FE00C9F0070085
:103F700012F10700C7F007003E0010000000B0007B
:103F80003E007800F8FF3200C2F007003E0040001B
:103F90002000B00009F10700801F78003E00780083
:103FA0001000B0000027780004F107001000B000F6
:103FB00000277800F00720003E006000AEF0070008
:103FC00008F10700002778004F0078000000060085
:103FD00042000000C5494E004B45590043F307001D
:103FE00000277800F5F00700002778000027780008
:103FF00030002000B5F007001000B000F9F0070015
:104000001000B10000277800F00720003E0060009B
:104010003E0040002000B000E8F00700000006006D
:1040200028000000C84B450059424F00415244004F
:104030002EF307001000B000002778001000B10038
:10404000DEF0070093F00700DCF007003E001000F0
:104050000000B0003E007800060032000027780023
:10406000D6F007003E0040001000B000D3F007007B
:1040700002003700002778003E00680000000600BC
:1040800030000000C6455800504543005400000071
:1040900000277800F00F20003E0060000027780025
:1040A00000002000002778003000200087F0070083
:1040B000CCF0070077F007001000B00075F00700A3
:1040C000002778000002200022F20700A2FF07006C
:1040D0000027780000277800F001200019F1070080
:1040E0006CF0070000277800F007200009F10700B6
:1040F0003E00600067F00700002778009000200075
:104100000AF107003E007000002778004000200000
:104110006EF00700A9F0070000277800400020009B
:104120006AF00700FBF007003E0060000000B000EE
:104130003E00780047003200002778000027780012
:1041400090002000F9F007000000B0003E00780069
:10415000180032003E00780000277800000220009E
:104160000027780080002000002778004000200011
:1041700056F0070091F0070000277800801F7800B4
:104180003E00780000277800700020003E006000AC
:104190003E00100000277800300020004BF00700A0
:1041A000002778004F0078003E0010007DF10700E6
:1041B000020037000027780010002000801F7800E0
:1041C0003E00780000277800801F78003E007800CD
:1041D00000277800FFF20700002778003000200059
:1041E0003AF0070075F007001000B00000277800D3
:1041F0004000200035F007007AF007000027780023
:104200003000200031F00700002778006BF0070035
:104210003E00400073F00700002778004F00780050
:10422000002778004F0078001000B10000277800C8
:10423000A4F007000000B0003E007800DFFF32006D
:104240003E0078003E007800002778000000200043
:104250004F0037000027780000277800F007200083
:10426000B2F007000BF00700002778008000200064
:10427000AEF007003E00700006F00700002778004F
:10428000C0012000A9F007003E0070000027780060
:10429000400020000DF0070048F0070090F00700F4
:1042A0003E0060000000B0003E00780014003200C4
:1042B0003E007800F7EF070040F007000027780085
:1042C000100020003E001000002778003000200081
:1042D000FEEF070043F00700002778008000200071
:1042E000BCF20700CAF50700002778008000200014
:1042F000B8F20700002778000000200024003700F3
:1043000000277800002778003000200087F00700A1
:10431000E0EF070000277800D000200083F00700BE
:104320003E007000DBEF070066F007003E00700003
:104330000000B0003E0078000B003200002778003B
:1043400030002000E1EF0700002778001BF0070095
:104350001000B0003E00400022F007000027780067
:10436000F0FF2F000A00370000277800A00020008F
:104370006EF007007AF007000000B0003E00780001
:10438000010032009BF507000027780000002000A4
:104390000000B0003E0078004CFF32003E00780084
:1043A0003E0078000000060094010000C451550052
:1043B000495400000FD020000027780000002000A2
:1043C000002778002CF2070001F0070030F2070008
:1043D000FFEF070028F2070010007800DEEF07006B
:1043E0000000B0003E007800150032000027780081
:1043F0004F80DE000000B0003E0078000400320074
:104400003E00780000277800A00320000B00370052
:1044100000277800200020004AF007000000B000CC
:104420003E007800030032000027780020022000C0
:1044300002003700002778008002200002003700C9
:1044400000277800E003200062F207008CF10700EB
:1044500000277800A4F10700100078000000B000E9
:104460003E0078000300320000277800F0052000AD
:104470000200370000277800E004200004FF070056
:1044800052F50700002778003000200081EF070078
:1044900000277800C9EF07003E0040001000B00080
:1044A000D0EF0700002778000000200079EF070018
:1044B000CCEF07001000B0008BF10700100078006F
:1044C0000000B0003E0078000800320000277800AD
:1044D000300120003FF20700E7FB070000277800CB
:1044E000100120003BF2070001003700E2FB07004B
:1044F000E7F10700100078000000B0003E007800EF
:10450000A00032000EE0200077F1070010007800D4
:104510000000B0003E00780009003200C4FE070031
:104520000000B0003E007800020032008AFE070062
:104530003E007800002778000000200002003700CD
:1045400000277800F0FF2F000000B0003E00780048
:10455000EDFF3200C8F10700100078000027780056
:10456000F0FF2F00F1EF07000000B0003E007800E0
:10457000200032008DF1070000277800801F7800AE
:104580003E0078002000B00010007800002778007E
:104590007FB89700100078003EEF07003DEF07005E
:1045A0003CEF07003BEF07000027780000002000E9
:1045B0000027780020002000A6EF070058F207002F
:1045C000A4EF0700002778007FB8970080EF07006E
:1045D000002778004F0078002000B0007CEF070033
:1045E000EFF107000027780000002000A2F107008B
:1045F00077EF070024FA0700052A2A002A2A20005C
:1046000026F10700BDF5070019F5070000F50700C2
:104610009FF107001000780000277800002778003D
:1046200010002000C1EF07000000B0003E0078003D
:104630000A00320014FA0700183A2000496E73008D
:1046400074727500637469006F6E2000494E4300F8
:104650004F4E4E0055452000217478000027780009
:104660000027780020002000B0EF07000000B00015
:104670003E0078000A00320003FA0700193A2000D1
:10468000496E730074727500637469006F6E200068
:10469000494D4D00454449004154450020217800D2
:1046A0000027780000277800300020009FEF0700E7
:1046B0000000B0003E0078000B003200F2F9070065
:1046C0001B3A200050524F00424C45004D452000FF
:1046D00050696C00652064006520520045544F000D
:1046E00055522000210D5400002778000027780043
:1046F000400020008DEF07000000B0003E00780071
:104700000B003200E0F907001D3A200050524F0024
:10471000424C45004D45200050696C006520640006
:1047200065732000444F4E004E4545005320210044
:1047300000277800002778004000200081EF070064
:104740000000B0003E00780008003200CEF90700FB
:104750000C3A20004552520045555200206E6F0021
:1047600020696C0079F60700010037003E007800F0
:10477000A0F4070095F4070000277800F0FF2F0051
:104780000F0037003CF10700100078004DEF0700E4
:104790000000B0003E0078000700320000277800DB
:1047A000F00420008BF1070000277800B0042000FF
:1047B00088F1070085F4070000277800000020003A
:1047C0000000B0003E00780002FF320000277800B1
:1047D000000020000000B0003E007800F5FE32002E
:1047E000000006001E020000C54142004F52540066
:1047F0000EE0200097F2070000277800000020005C
:104800000027780031F10700F1EE0700002778005B
:1048100027F10700EEEE070000277800BFF0070041
:10482000EBEE0700C3F00700E9EE070067F40700AE
:1048300095F90700262A2A002A2A2000494E54000A
:104840004552520055505400494F4E00204C6F00C5
:104850006769630069656C006C652000284142004F
:104860004F5254002920210058F4070061F407003A
:10487000D0FE07000000060000277800600320003B
:1048800000277800801F78003E0078001000780034
:10489000002778004F0078000027780010002000E3
:1048A00098F007001AF00700C9EE07000040060064
:1048B000002778006003200000277800801F780020
:1048C0003E00780010007800002778004F00780044
:1048D0000027780010002000BAF007000CF0070055
:1048E000002778004008200000277800801F78000B
:1048F0003E007800100078000027780070FF2F003D
:104900003E006000002778004F007800B0EE0700FE
:10491000E7F0070010007800EAEE07000000B000A2
:104920003E0078008C0032006FF007001000780025
:104930000000B0003E0078002C0032006AF0070052
:1049400000277800801F78003E0078001000780073
:104950001000B10000277800002778004F00780091
:104960009BEE0700D7EE07000000B0003E00780085
:104970001E003200DDF00700002778008FEE0700F0
:104980001000B00000277800F00720003E00600013
:1049900040EE07001000B00088EE07003DEE070073
:1049A000E2EE07000000B0003E0078000300320095
:1049B0003E0078003E0078000C00370000277800A9
:1049C000D000200000277800300020003FEE0700D4
:1049D0000027780079EE07003E0040002000B0007C
:1049E00080EE070024EE07007EEE0700B7F0070018
:1049F0001000780079F00700100078000027780098
:104A00000000B0003E0078005100320021EE0700A7
:104A100020EE070010007800B8EE07000000B0009C
:104A20003E0078004500320066F007001000780074
:104A300018EE07002000B000100078000027780072
:104A40004F80DE00801F78003E0078003E0010009E
:104A500000277800000024003E0060000027780056
:104A60004F0078003E007000BDEE07000000B0006F
:104A70003E00780017003200002778001000780010
:104A800092F0070052EE070000277800000028008F
:104A900000EE07002000B0009DEF0700002778001F
:104AA0004280BF00002778007FF89700004EB200D8
:104AB00042E0B7003E007800F6ED070003F807007B
:104AC00042E0B7003E007800F2ED07007FF00700FB
:104AD0003FEE07003BF00700811F7800821F78003F
:104AE000100178009E0078008180E8001100E0004D
:104AF0000B003B00210090000000E00008003200A5
:104B000002003B00110010000300370000004100CC
:104B10000001EB00A200980000F0A10080087800DE
:104B20003E0078004F017800CF0078002000900010
:104B30000027780063EE07000200370000277800A6
:104B4000F0FF2F000000B0003E007800AFFF320001
:104B50003E0078003E0078005CF00700100078000E
:104B6000002778002000200064EE07000000B0005D
:104B70003E0078003700320027F007000027780059
:104B8000801F78003E007800100078000027780031
:104B90004F0078002000B00010007800BDED070045
:104BA000BCED07003E0070000000B0003E00780041
:104BB000260032000027780000002000002778003F
:104BC00015F0070000277800801F78003E0078006D
:104BD000FFED0700002778004F0078002000B000AC
:104BE000FBED0700CDEF0700100078000000B000DB
:104BF0003E0078001200320000277800F007200005
:104C00003E006000002778004F0078000027780001
:104C100000F82F003E0060003E00400000277800B2
:104C20004F0078003E00780093ED0700801F780069
:104C30003E007800801F78003E00780002003700B8
:104C40003E0078003E007800020037003E00780009
:104C50003E007800DEED07000040060000277800E7
:104C60006003200000277800801F78003E00780055
:104C700010007800002778004F00780000277800A7
:104C800060222000CDED07000027780040082000BA
:104C900000277800801F78003E0078001000780020
:104CA00000277800F07F2F003E006000002778008A
:104CB0004F007800C6ED070085EF07000027780059
:104CC000801F78003E0078002000B00010007800BF
:104CD000002778004F007800100078006DED070085
:104CE0006CED07003E0070000000B0003E00780050
:104CF000020032004DF90700460037003E00780000
:104D00003E007800002778001000B1000000B000DD
:104D10003E0078003200320000277800002778003B
:104D20003001200001EE07005AED0700002778004F
:104D300010012000FDED07003E0070000000B000F3
:104D40003E00780007003200002778003001200084
:104D5000F6ED0700E5EF07002008B000A1ED070021
:104D60001E003700E1EF07000027780093ED0700F1
:104D70001000B00000277800F00720003E0060001F
:104D800044ED07001000B0008CED070041ED070076
:104D9000E6ED07000000B0003E007800040032009D
:104DA0003E0078003E0078003E0078000B0037009F
:104DB0003EED0700002778003000200043ED07009B
:104DC000002778007DED07003E0040002000B00085
:104DD00084ED070028ED070082ED07000D00370085
:104DE000002778003E00680000277800403F22003E
:104DF00089EF070000277800801F78003E007800C8
:104E000073ED0700002778004F0078002000B00005
:104E10006FED07006EED0700004006001C03000068
:104E2000D15449004D455200315F55004152540064
:104E3000315F49004E49540000277800F0E7230015
:104E4000002778002010200061ED0700002778007F
:104E50000000280000277800401020005CED0700CB
:104E60000027780020022000002778008022200000
:104E700057ED070000277800000020009BEF070097
:104E800053ED0700002778008000280000277800F5
:104E9000002220004EED070000277800004020008F
:104EA000002778002022200049ED07000027780025
:104EB00080802000002778004009200044ED070092
:104EC00000277800000020000EEF070040ED0700EB
:104ED000000006005C000000C55445004D504F0026
:104EE00038EF0700100078000140FE00E9EC0700F1
:104EF00034EF070010007800002778003000200011
:104F0000F2EC07003E0010007CED07000000B0004E
:104F10003E007800F4FF32003E0078003E0078004A
:104F20000000060028000000C5464F00525448000B
:104F3000D5F70700C90D45006E747200657A200030
:104F400064616E0073206C0065206D006F6E6400FC
:104F500065206400752046004F525400480D0D0036
:104F600020202000202043006F70790072696700C4
:104F7000687420006A7062002E666F0072746800A8
:104F80000D0D200020204D00696372006F20460047
:104F90004F525400482070006F7572002050490035
:104FA00043323400460D20005665720073696F006D
:104FB0006E2031002E323200202064007520310036
:104FC000362F3100312F3200303134000D202000D7
:104FD00068747400703A2F002F6A7000622E6600A9
:104FE0006F727400682E6600726565002E6672002E
:104FF0002F0D2000206A7000625F66006F727400DF
:105000006840790061686F006F6772006F757000AB
:10501000732E63006F6D0D000D205100756520002B
:105020006C652000464F520054482000736F6900A1
:10503000742061007665630020544F0049210D0003
:105040000D210D000000060092000000C6464F0032
:105050005247450054000000D6F407008DEC0700CD
:105060008CEC07003E0070000000B0003E007800AD
:105070001D00320087EC070086EC0700002778004F
:10508000000020000027780020002000F1EC07003D
:1050900080EC07007FEC070041EF0700A0EF07005E
:1050A000ECEC0700C1EE070000277800801F7800B5
:1050B0003E007800C6EC0700002778004F0078001B
:1050C0002000B000C2EC070000277800F00F20009D
:1050D00000277800F0FF2F0023EF0700B6EF07004E
:1050E0005CF00700020037003E0078003E007800C8
:1050F0000000060056000000CE5445004C45430019
:105100004841520047454D00454E5400E8EE070027
:1051100000277800801F78003E007800100078009B
:1051200000277800F0FF2F00002778007FB8970055
:10513000A7EC0700801F78003E0078000027780069
:1051400080BB200068EE0700A1EC07000027780074
:105150004F007800002778004F0078009CEC070093
:105160000000060038000000C94445004D415200CF
:105170005241470045000000A0DA200020A0B700FF
:105180000FD020000EE020003DEE07000027780041
:10519000005020000027780000002000EDED0700FF
:1051A0000027780010002000D7EE070088EC0700E9
:1051B0000027780080A5200035F007001EFF0700BB
:1051C0000CF307000027780000002000002778007B
:1051D0000010200052EF07002EEC07002DEC070016
:1051E0000027780000002000002778002000200021
:1051F00086EC070027EC070026EC070048EF0700C5
:10520000801F78003E00780000277800F00F200013
:10521000C6EC0700002778004F00780000277800D0
:10522000F0FF2F00C1EC07003E0060000000B0005E
:105230003E007800EAFF320016EC070015EC07008C
:10524000D7EE070013EC070000277800500020007D
:105250001EEC0700B5EC07000EEC070000277800F5
:105260005000200019EC0700B0EC07003E00600081
:105270000000B0003E007800050032003E007800DB
:105280003E00780000277800F0FF2F00690037000B
:1052900000EC0700FFEB070000277800000020006B
:1052A00000277800200020006AEC07001CEF0700B0
:1052B000F8EB07000000B0003E0078000A00320062
:1052C0003E0078003E0078000027780000002000B3
:1052D00000277800200020005EEC070000277800FF
:1052E0000000200053003700801F78003E00780047
:1052F000801F78003E007800E6EB0700E5EB070032
:10530000002778004F007800002778004F007800D1
:1053100050EC0700DFEB07004F80DE000000B0001C
:105320003E0078000C0032003E0078003E0078001D
:1053300000277800000020000027780020002000CF
:1053400044EC0700002778000000200000277800C8
:10535000F0FF2F0034003700CEEB07000027780065
:1053600070002000D9EB070070EC0700C9EB0700C4
:105370000027780070002000D4EB07006BEC0700DA
:105380003E0060000000B0003E0078000A003200DD
:105390003E0078003E007800C4EB07003E00780035
:1053A000C2EB07003E00780000277800F0FF2F00D6
:1053B000002778001C003700B6EB0700B5EB0700AC
:1053C000002778000000200000277800200020003F
:1053D00020EC0700D2EE0700AEEB07000000B000A3
:1053E0003E0078000E0032003E0078003E0078005B
:1053F0003E0078003E007800002778000000200082
:10540000002778002000200012EC07000027780019
:105410000000200000277800F0FF2F000200370076
:1054200000277800000020000000B0003E00780057
:10543000B7FF32000000B0003E00780081FF32006C
:1054400094EB070093EB0700D8ED070000277800E6
:10545000801F78003E007800DDEB07000027780011
:105460004F0078002000B000D9EB070089EB07005F
:1054700088EB0700AAEE0700801F78003E00780046
:10548000002778001004200028EC0700002778008F
:105490004F0078000027780050CC240023EC070050
:1054A0003E0060000000B0003E00780020003200A6
:1054B000002778000000200000277800200020004E
:1054C000D2EB070073EB070072EB070094EE0700C6
:1054D000801F78003E0078000027780050042000EC
:1054E00012EC0700002778004F00780000277800B2
:1054F000E03424000DEC07003E0060000000B00026
:105500003E007800070032000027780000002000ED
:105510000027780020002000BCEB070043F70700BD
:10552000020037003E0078003E007800020037009D
:105530003E0078003E00780026F207007CFE07005F
:105540002CF107009BFB070000000600FFFFFF0097
:00000001FF
